:020000040000FA
:10000000F128FF3FFF3FFF3F8C00030E8D008E0A5B
:1000100003198E036400980A0319970A0319960FAF
:100020001828FC3096006C309700793098009114B5
:100030000D0E83008C0E0C0E0B1109008207C134CB
:10004000BE34BE34BE34C134FF34DE348034FE34BA
:10005000FF34DE34BC34BA34B634CE34BD34BE34AE
:10006000AE349634B934F334EB34DB348034FB34BF
:100070008D34AE34AE34AE34B134E134D634B6342B
:10008000B634F934BF34B834B734AF349F34C934DC
:10009000B634B634B634C934CF34B634B634B534E5
:1000A000C334FF34C934C934FF34FF3407309900F6
:1000B00012309400950192019301FC3096000034B7
:1000C000003066001730650000340B118B178B165B
:1000D00081016400D83062008101003405081106F6
:1000E0001039031900349106111A00340E088F00DC
:1000F0008E019301920110080F02031C8328023C19
:10010000031C900A0034023E031C900300340530A7
:100110001206FF300319A9280310130D8207140ECD
:100120009A2814089A280A309A28150E9A28150831
:100130009A2800340F399A009A079A079A079A0763
:10014000031DA6289308FF300319A92812081A07CF
:100150001E2086000310100CF43EB620920A0630D2
:100160001206031D00349201930A00349B009B0B7E
:10017000B72808000508190607390319003499063D
:1001800064309A00FF30B6209A0BC228191DE4286B
:10019000991CCD28191CD32800340A309A00E42079
:1001A0009A0BCF280034123014060319DE280730CA
:1001B00014070730831C0130940700340130940089
:1001C0000034911C00349110073015078318EA2879
:1001D000950A0034950060301506031D0034950122
:1001E000D3285620602065206E208720BA20E12089
:0401F000F428FF3FB1
:02400E00F53F7C
:00000001FF
